:0A00000002000E7400C0E0C0E03200
:10000B000217F675817402184CF183E4F560800BCE
:08001B007F2EC1BE53D8EF3265
:0B00260090E60174CAF0227F1CC1BEEE
:0200330080EA61
:0C004300020200F13244E0FD7F2C61025B
:10005600EB9FF5F0EA9E42F0E99D42F0E89C45F000
:1000660022E8600FECC313FCED13FDEE13FEEF1355
:10007600FFD8F122E8600FEFC333FFEE33FEED3316
:10008600FDEC33FCD8F122E6FC08E6FD08E6FE08A6
:10009600E6FF22ECF608EDF608EEF608EFF622A4E7
:1000A6002582F582E5F03583F58322D083D082F868
:1000B600E4937012740193700DA3A393F8740193E3
:1000C600F5828883E4737402936860EFA3A3A38028
:1000D600DF90E682E044C0F090E681F043870100BD
:1000E60000000000227400F58690FDA57C05A3E5BE
:0600F60082458370F9222F
:100100001201000200000040B40411464002003F0A
:10011000330109022000010100C0000904000002AF
:10012000080650000705020240000007058802404B
:10013000000009022000010100C0000904000002C3
:1001400008065000070502020002000705880200A9
:1001500002000403090418033000300030003000AE
:1001600030003000300030003000300030002A0312
:100170004300790070007200650073007300200076
:100180004400690073006B00200032002E00340030
:1001900030005200430039000A060002000000400F
:1001A00001008E6D8F6E90E600E054187012E56EBF
:1001B0002401FFE4356DC313F56DEF13F56E801563
:1001C00090E600E05418FFBF100BE56E25E0F56ED9
:1001D000E56D33F56DE56E156EAE6D7002156D4E05
:1001E00060051200EB80EE228D828C83A907E0F57A
:0F01F000F0E7B5F007A309DBF57F00227F0122BE
:0A020000021C65D1BEEF54F0FF228E
:03020C00021D458B
:03021000021701D1
:10021400021B6E437970726573732053656D6900B8
:100224000B0803052400000000023A000303000346
:1002340011000312000520000521000526000553C6
:10024400020628000629000727000A02123F0311AC
:10025400013F0202020702030207FEFEFFFF07112D
:10026400013F00000036020302070404163F031195
:100274003F000000060100010700FDFDFFFF08111B
:10028400043F00000000000106010801061C0101F2
:1002940002070100020302022600FFFBFAFAF8FB40
:1002A400FBFF09091209002D363F08011301010261
:1002B40001070100010000262600FFFBF8FBFBFB01
:1002C400FFFF0909091B002D363F75080C301C0679
:1002D4007FD07E0731A2301C0D1217ECC21C7F5A4E
:1002E4007E0031A2800A7D047F1C71027F3251FAA4
:1002F4007FE87E0321A27E0031A2E4FD7F1CE5BBE2
:1003040030E7FB90E6C0E4F1E2EDF0E5BB30E7FB5B
:100314007580BE221146E52A54FE45296013300437
:10032400067D017F247102F17D756B01756C00807F
:100334003B302316F18AC333CE33CED8F9FDAC0655
:10034400E52C24FFE52B3401800EF18AC333CE3330
:10035400CED8F9FDAC06E52BC3132DF56CE43CF5C2
:100364006B300402F17DAD6C7F247102300410AD5A
:10037400097F267102E4FD7F2871027F2A7102AD94
:100384000C7F267102AD0B7F287102AD0A7F2A71A2
:100394000220040DF132FFE50944E04FFD7F2C718A
:1003A40002E4FCFDE50C256CF50CE50B356BF50B57
:1003B400ED350AF50AEC3509F509AE6BAF6C229000
:1003C400F00EE0540FF5611146111BEF20E7FA7DA2
:1003D400FE7F2871020D7F2A71023020047D018086
:1003E40002E4FD7F2271027DA07F2E7102112D8F08
:1003F40062E56254C0FFBF40F4E56230E004918BD3
:10040400D322856163E563C3940C5011740F256393
:10041400F582E434F0F583E4F0056380E8759AF03E
:10042400759B0FE5BB30E7FB90E6C0E4F07580A058
:1004340075630690E67BE0F564E5BB30E7FB90E688
:100444007BE090E6F0F0A3E564F0D563E62020209D
:10045400E58030E0FB112DEF30E002D3227562809D
:10046400E5625490641060087F1CD1BE8F6280F0F6
:10047400918BC322E4F50990F010E0541FF50AA310
:10048400E0F50BA3E0F50C90E6917480F02290F077
:100494000DE0F55E6536702C301A29C21A7F0D7B8B
:1004A4000B7D0F7CF031E8EF7011D154E433F55F2C
:1004B400121D18918BAF5FB1E5A1AEF183E4F55F36
:1004C40011268002C21A121CFDE55EB53603D380E4
:1004D40001C3407CE55E75F00AA42441FD7F371218
:1004E40018F7255EF8E6F520855E363005207C0297
:1004F4007D627B0CB1B67C027D827B0C7F20B1B81F
:1005040090E61B7404F090E618F011268042F18303
:1005140090E618F0E53B30E10E7C027D527B0CB195
:10052400B67C027D728027E53B30E01A7C027D5266
:100534007B0CB1B67C027D72F19390E4007406F0FA
:1005440090E420F0800A7B0CB1B27C027D6EF193C2
:1005540090F00FE0B4FB1690F00CE020E70F918BC5
:10056400AF2CAE2B121E3BE4FFB1E5803D201F05EE
:10057400120D84701A755A03300305120F9C8006FD
:10058400120A39E433FFB1E5E5BB30E7FB801875A7
:100594005A023003051213628006120DEBE433FF96
:1005A400B1E5E5BB30E7FB7580BE755A01227C02DC
:1005B4007D4E7F007A007EE48E638F64EEF59AE5CB
:1005C40064F59BEB1BAE0270011A4E60130DEDAE89
:1005D4000470010C14F5828E83E090E67BF080E3D6
:1005E400228F60C22220225590E6A6E020E3F6E0A6
:1005F40020E0F21211E5E560B4020890E6A374016C
:10060400F0D218E4F59E90E67C7455F07453F074BF
:1006140042F07453F0E556F0E557F0E558F0E5592B
:10062400F0E52CF0E52BF0E52AF0E529F0E560F0A3
:1006340090E69CE4F0A3740DF0D22280A830180A4E
:1006440090E6A6E030E2F9121930301A02F1B22233
:10065400120D84605FC2223004047D2580027DC8AF
:100664007F2E7102E531FFE5321217B51216C17003
:10067400051216EA601090E6D0A3E06002D21911C8
:1006840014120A19D222111BEF30E007D223120DE3
:10069400918006302207E4F5081114D322E4B53220
:1006A4000EE531B40109F1A9121F57F52980A112F1
:1006B40016B1809CD21A1114C322E5BB30E7FB901B
:1006C400E6C07410F1E2E0FFE5BB30E7FB90E6F230
:1006D400E0FF7580BE227F0551FAF15411467D1F5B
:1006E4007F3E71027F2C5103A201E433FEC454F017
:1006F40044E0B50703D38001C350327F2AD1BEBF83
:10070400EB097F28D1BEBF1402D203200103D2001B
:1007140022300312F165112DEF30E611121F74D24D
:1007240000A22292AF22111BEF6002D20022A2018A
:10073400E433C454F0228F6B1146F156AD6B7F2421
:1007440071027D037F2271027DEF7F2E7102800290
:100754001146112DEF20E7FA112DEFC330E001D33C
:10076400221146F1563003047DA180027DEC7F2ED8
:100774007102E58030E0FB80D9E4FD7F24610290C2
:10078400E61B7405F0227E00E52A54017807227BDB
:100794000C7A007F207EE4A1BCF15490F011E0F5C6
:1007A40009A3E08181D22371188E318F3222AF0CDC
:1007B400AE0BAD0AAC09780F11997817118D121E82
:1007C40001F1A990E6C77436F074021217E474D0EC
:1007D400F090E61B740DF090E60174C6F022F0EF81
:1007E4004480F58090E6F1227F2AD1BEEF7D00FCA3
:1007F4007F28D1BEAE042290E61BE0FB54F7F07FC5
:10080400007E021117E5BB30E7FB7580BE90E61B46
:10081400EBF022AD07AC06E5BB30E7FB90E6C07415
:1008240001F00DBD00010C121F6275BB07228F631E
:10083400E563B42F23E4F52C90F016E025E0FEA345
:10084400E07C002400FFEC3EFEEF25E0FFEE337871
:100854002AF608A607E4F5297F0D7B0A7D0F7CF0B4
:10086400121D2BF1F77817120099E56324F870052F
:10087400120478800312079DB18470024117D223B9
:100884001203188E658F66E53C600DE563642F6086
:1008940007121558700221B230040DE563B42F0419
:1008A4007D42800F7D24800BE563B42F047D40805E
:1008B400027D207F2E120302E563642F701B120752
:1008C400565009D223B1911216B1D322E4B566076A
:1008D400E565B40102410B411212002DEF20E7F946
:1008E400E5661566AE65700215654E608B12001BD9
:1008F4008F64E564548864086008E5645481FFBF2C
:1009040001EBE56430E022D223B191E56430E315D4
:10091400E4FDFC7F201206BE0DBD00010CE4B5050C
:10092400F2ECB401EE5119D322E52E6440452D704A
:10093400057568088003756801E4F567E567C39584
:1009440068503CB1846038B176AE2DAF2E12124699
:100954001200564006AE2DAF2E8004AE2BAF2C8E67
:10096400698F6A1117E5BB30E7FBE56990E69CF0F7
:10097400E56AA3F0AE69FFFB12151C056780BDE5AF
:1009840067C39568400EE56A652E7004E569652DB8
:10099400700201E412001BEF30E3077F201206BE51
:1009A40080F290E6A6E030E2F912111E01E412078B
:1009B400C73004047D2580027DC87F2E120302E522
:1009C40065FFE5661217B5120783E4F5681216BBD6
:1009D40070051216EA600D90E6D0A3E06002D21909
:1009E4005119C21A120756500DD223B191E508705D
:1009F40003121E18D322E53360021533D21AE4B56C
:100A0400660CE565B40107121F57F529017C12161F
:100A1400B1017CC322B184601B20190E90E6A6E0CC
:100A240030E2F990E69CE4F0A3F090E6A6E030E230
:100A3400F912193022C21990F00FE0F5601200B1DA
:100A44000BB3000BC5030BB3040B19080A78120B84
:100A5400A4150C701A0C041B0C041E0B4D230B4D17
:100A6400250B19280B272B0B192F0BA4550C705A87
:100A740000000D6C12048BB176300526E4F59E75EA
:100A8400612C90E67CE4F0D561F890FC01E04480B0
:100A9400F07C027D177B0D7A007F087EFC1205BC7A
:100AA40080691207651207FB7B007A017D007F00D5
:100AB4007EFD121FAF75612C90E67CE4F0D561F8E1
:100AC400759E08E4F561E56164012436F582E43439
:100AD400FDF583E090E67CF00561E561B418E790EC
:100AE400E67C7430F090FD92121FC87430F090FDD3
:100AF40094121FC890FC01C083C082E0FF90FD00E7
:100B0400E05480FEEF4ED082D083F090FC04741F3A
:100B1400F07F2C8100750802E508B40204AF60017F
:100B2400328021121FC0701C12079DD22312031899
:100B34007D707F2E1203021207565006D223B19104
:100B4400D322C32212048BA17275610812048B751F
:100B54000802B176E50864027044F59EE560B423AA
:100B64000D90E67CE4F0F0F07408F075610C90E60A
:100B74007CE53DF0E53EF0E53FF0E540F0E560B4AE
:100B840023057402F0800590E67CE4F090E67CE4B2
:100B9400F07402F0E4F0AF61FE12159BC322A1725F
:100BA40012048B750802E508B40202C322D322B1F1
:100BB4007E60025119750802E508B40202C322D30B
:100BC4002212048BB176E4F59E90E67C7470F0E416
:100BD400F07B10FA7D017CFC7F027EFC1205BC9048
:100BE4000224121F39759E07740AF0759E0C900238
:100BF40025121F40900226121F397F127E00A16425
:100C040090F013E0F561B17E6002511912004612B2
:100C14001FC06002D322120756E560B41E0DE561C1
:100C240030E0047DDE80157DDF8011E5615403FF33
:100C3400BF020E300504D21E80077DED7F2E120305
:100C44000212075612001BEF30E01FD223B1918F1E
:100C540062E56230E202A167E56230E10BE56154CE
:100C640003FFBF020375080AD322C32290F011E0E8
:100C7400543FF56112048BB176E5616405601DE5AE
:100C840061643F6017E56164016011E561640860B7
:100C94000BE561641B6005750801A17290FC00E41A
:100CA400F07B63FAFD7F017EFC121FAFE560B45A4E
:100CB4001A90E67CE4F0E561B43F057436F08006F2
:100CC40090E67C7412F0759E088013E56190E67CD2
:100CD400B43F057433F08003740FF0759E04E5612E
:100CE40064056006E561643F70317405F1EF90E6D8
:100CF40080E090E67C30E70674FFF0F08006742E06
:100D0400F074E0F090E67CE539F0E53AF07402F036
:100D1400E4F0E537F0E538F0E4F0F0E561641B60F9
:100D240005E561B43F0F741B121FB8E4F004F074BE
:100D340008259EF59EE56164016005E561B43F09FF
:100D44007401121FB8259EF59EE56164086005E5EF
:100D540061B43F087408F1EF259EF59EAF9E7E00B6
:100D640012159B750802C32212048B7508075119CA
:100D7400D32290E6A6E020E3F92290E6917480F075
:100D8400AF2CAE2BAD2AAC29EC4D4E4F227F221254
:100D940006BEEF7005750802804CEF30E705E4F5F8
:100DA400088043EF30E105750803803AEF30E5052C
:100DB40075080B8031EF30E4057508068028EF30A4
:100DC400E60A302302801275080D801AEF30E30220
:100DD4008011EF30E20D3023057508058008750891
:100DE4000480037508072290F00FE0FF24EB6026CF
:100DF40024EB600E24FC600A24D96021244B600299
:100E0400C188750802E508B402030213A6B17E6026
:100E1400031211FDD3227F057E001201A2C222809B
:100E240052B184605320225090E6A3E020E2F2F114
:100E340094FF121246D3120056400CF194FFE4AB17
:100E440007AA06F9F8800AF1F7AB07AA06A905A8CC
:100E540004C3E52C9BF52CE52B9AF52BE52A99F593
:100E64002AE52998F529F194652E7003EE652D6025
:100E740002D22212048B80A9750802E508B402028A
:100E8400C322D322B17E60031211FD750807D32259
:100E9400121F84C223C224E56130E002E16E3023D4
:100EA40002E16EB1847002E16EB176C3E567952EFE
:100EB400E566952D4002E14D302302E14DB1847089
:100EC40002E14DE56345627032D22512155F8F61F0
:100ED40012001BE56130E0028014E56120E306D2D4
:100EE40023C22480647F241206BEEF20E106D223AD
:100EF400D22480551207EC8E628F63121F9495637F
:100F0400EE956250028004AE62AF638E648F65E535
:100F14002A45297019C3E52C9565E52B956450067F
:100F2400AE2BAF2C8004AE64AF658E648F65AF6565
:100F3400AE641117C3E5639565F563E5629564F5E1
:100F440062121516121FA2C1AFE5BB30E7FBE566BE
:100F540090E69CF0E567A3F0C3952EE566952D50C9
:100F640002D219E4F566F567C19B202305E58030BC
:100F7400E0FB12075650037F012212002DEF20E3FD
:100F840006E563456260037F0222A224E433FF2264
:100F940090E690E0FEA3E022C219E53C6004D22072
:100FA4008002C220E52C452B700CE52A45297006E9
:100FB400C222C2208002D2221217DC600551197F9E
:100FC400012220220C12001BEF7F0030E31C7F0261
:100FD40022302007121D4E8F608004D1948F60B19F
:100FE4008460055119AF6022AF602290E67CF074F2
:100FF4000AF022AF2CAE2BAD2AAC292212076512BF
:10100400001BEF30E3F9121F7420034C7E007F565F
:1010140074022FF58274E03EAD82F55D8D5E74003E
:101024002FF58274E03EF583E0C31314F55FE4FF0B
:10103400EFC3955F503274142FF582E434FCF583CA
:10104400E0F560855E82855D83F00F7402255EF5B0
:101054005EE4355DF55D80D874002410F58274E09B
:101064003400AF82F55D8F5E90FCA7E030E207D2DA
:101074000490FCC88005C20490FC78E0F540A3E02D
:10108400F53FA3E0F53EA3E0F53D90FC6DE0F537B8
:1010940090FC6CE0F53890FC6EE0F53990FC70E063
:1010A400F53A90FC80E0F53BE4F53C90FC6AE030D6
:1010B400E21DE4F55D90FCB0E05414F55DE55D30AF
:1010C400E405753C448008E55D30E203753C4290DC
:1010D400FCA6E0F55C311EA22292AF200522E53C7D
:1010E4006003FF8018E53B30E108E53C70127F0C9B
:1010F400800BE53B30E009E53C70057F0B12073AB5
:10110400C3E5409401F540E53F9400F53FE53E9486
:1011140000F53EE53D9400F53D2290E6047408F0A8
:101124002290E6827445F0E030E63B90E680E044AD
:1011340008F0F183311E31E590E6C37480F090E647
:10114400C2E4F0F5B2C2AF7F1EFE1201A290E682A5
:101154007451F01200D790E6827445F07F1E7E0031
:101164001201A202000390E6C3E4F090E6C2747791
:10117400F075B2BE2290E6707401F07580BEC2882C
:1011840012002690E6007414F090E603E4F0312592
:1011940090E6C1E4F090E6CEF090E6C8F090E6CC9C
:1011A4007403F090E60C7401F090E61274A0F090D1
:1011B400E6187405F090E630E4F0A3F090E61574B8
:1011C400E0F012078390E6147422F090E613F09096
:1011D400E611F090E610F090E60B7402F031E52190
:1011E4001EE58E54F84405F58E90E6047402F01260
:1011F400048BF0F0F0538EF822E5AA30E007E4F512
:1012040069F56A8002B17D5142D3120056402E9096
:10121400E6A3E04401F0F1D590E6A3E030E00675E2
:101224006904756AD2E5AA30E007E4F569F56A80D5
:1012340002B17D5142D31200564002D1F922AE6967
:10124400AF6AE4FCFDAB2CAA2BA92AA82922121F01
:1012540084C222C223F5683022026137120D8470E1
:1012640002613790E6A3E0540570ECF179FE90E654
:1012740090E05EFEA3E05F4E6002D22390E691E42C
:10128400F0F566F567D3E52E9567E52D956640C7BD
:101294002022C4120D8460BFE56245617033D225FB
:1012A400B15F8F6312001BE56330E007756801D2FC
:1012B4002280A4E56320E307D222E4F56880127F4C
:1012C400241206BEEF30E10280131207EC8E618F08
:1012D40062AE61AF625146C31200565007D2227506
:1012E4006802415B121F949562EE9561500280047E
:1012F400AE61AF628E648F655146C31200565006CC
:10130400AE2BAF2C8004AE64AF658E648F65E5654B
:101314004564600BE5652401FFE43564FEB136B134
:1013240016C3E5629565F562E5619564F561121F82
:10133400A24189C225B15F8F63E56320E306E562BC
:10134400456160057568028008E56330E0037568EF
:1013540001120D84600520230231FDAF68227560FF
:1013640001C220E53C601690F00FE024D66008240A
:1013740080600424A07004D2208002C220F1DC60CA
:1013840012E4FFFEFDFC5149D3120056400231FD28
:101394007F0122120D847003AF6022302002C13B12
:1013A4004152E4F560EF640A600512079D80031260
:1013B4000478E4FF7E02FDFC5149C312005650023A
:1013C400C322E53C6006B1587002B1D4E4FF7E024A
:1013D400FDFC5149C3120056500281F7C223120387
:1013E400188E618F62E53C605CB158705812002D14
:1013F400EF20E7F93004047D3580027DCA7F2E1288
:101404000302E4B5620CE561B40107E4FBFD7F016E
:101414008008E561FFE562FDE4FBF195D1CAD1C125
:101424007004D1EA600231FD12001BEF30E002A12A
:101434000DE4B5620CE561B40107121F57F529806C
:101444008BD1B18087E53C6007D1F1F564120026A9
:101454003004047D3480027D307F2E120302E56265
:101464001562AE61700215614E700261D012001BEC
:101474008F60E56054886408600AE5605481FFBFAA
:1014840001EB806FE52E6440452D7005756408807E
:1014940003756401E4F563E563C39564504690E61F
:1014A400A3E020E2F9120F94FDEDFBAA06C3952EEA
:1014B400EA952D5020E4F0EB2401FFE43AFEB13626
:1014C400E56375F040A42BFFE5F03AFEFAC3E52C82
:1014D4009FB122801E90E691E4F0AF2EAE2DB1367E
:1014E400056380B3C3E52C9400F52CE52B9402B17D
:1014F40027816212002690E6183005057404F080F6
:10150400037405F0E56030E007C223120D91D32285
:10151400C322AE64AF65AB07AA06C3E52C9BF52CCA
:10152400E52B9AF52BE52A9400F52AE5299400F594
:101534002922AD07AC06756900756AC8E5BB30E7BA
:10154400FB90E6C0E4F0121F6290E6D4E4F0E5BB41
:1015540030E7FB22E52B5401452C22E58030E0FBEB
:1015640012075612002DEF30E00122302505EF302E
:10157400E30622EF20E301222290E6ABE0FEA3E0A3
:101584007C002400FFEC3EFE90E690E0FCA3E02FFC
:10159400F56AEC3EF569228E638F645146C31200EE
:1015A400565006AE2BAF2C8004AE63AF648E658FAD
:1015B40066E56590E69CF0E566A3F0AE65FBB11CBC
:1015C400F1795565FEE5665F4E6002D219020A198B
:1015D400E4F567F565F566E567C394045029AE65DF
:1015E400AF665146120056401E90E6A3E020E2F991
:1015F40090E691E4F0F5680567E52E2566F566E565
:101604002D3565F56580D090E6C77470F07408F1E7
:10161400E47411F0E53C90E6CDB442057404F08026
:10162400037402F090E6D27401F090E6017486F03F
:1016340090E6187411F022E52C2401FFE4352BFE0A
:10164400E4352AFDE43529FC121E0AB1D4F18FD108
:10165400CAD1F1F561D1BB7008D1EA7004D1B2806E
:1016640038120D84600231FDD1C1702DE52C540176
:10167400F52CE4D1B4A3A3E025E0FF0582D58202D2
:1016840015831582E033FEE52C4FF52CE52B4EF542
:101694002BE52AF52AE529F52912075650037F017F
:1016A4002212001BEF7F0030E3027F0222E4F52CBC
:1016B400F52BF52AF5292290E60174CAF090E6CEBE
:1016C400E0FEA3E04E22E4F56590E6C67483F09054
:1016D400E6D4E4F0E58030E0FBE5BB20E702F183EB
:1016E40090E6C6E4F022A3E0FEA3E04E2290E618C2
:1016F4007401F0E42231E590E6A3E4F022C0E0C0F6
:10170400F0C083C082C0D075D000C000C001C00248
:10171400C003C004C005C006C007121B4DF583A357
:101724007402F0121B58F583A37407F0752D00752D
:101734002E4090E6367480F0A37460F0121BF431EE
:101744001ED1F990E6A6F0F530F52F5391EF75A16F
:1017540010E55A6005C2AF120003D007D006D005C9
:10176400D004D003D002D001D000D0D0D082D08316
:10177400D0F0D0E032E52E24FFFFE52D34FF229097
:10178400E6C6E4F090E6F574FFF022AB64AD63AF17
:1017940062E5BB30E7FB90E6C0740BF07580B09057
:1017A400E6CFEFF0E4F56BA3EDF0E4F56BA3EBF01B
:1017B40022FDE4FBF19590E6C67482F075BB07E563
:1017C4008030E0FBE5BB20E702F18390E6C6E4F05D
:1017D400227F647E000201A21203C3E433F5602277
:1017E40090E6C9F090E6CB2243B280C287F1D5D20D
:1017F4008722C0E0C0F0C083C082C0D075D000C0D2
:1018040000C001C002C003C004C005C006C007AFC9
:10181400351535EF7005153475353D12112590E6F3
:1018240080E02086054408F0800354F7F0D007D008
:1018340006D005D004D003D002D001D000D0D0D03F
:1018440082D083D0F0D0E0321217839126D2E843BD
:10185400D82090E668E04408F090E65C7439F0C261
:1018640021D21DC21E1202CEE521702AE522702665
:1018740085555BE55BC3940250EEE4F520E55B24FB
:10188400FF92011206DA30000974212555F8A620CA
:101894000555055B80DDE4F55BE55BC39555502498
:1018A4007421255BF8E6F520300015121000E55B85
:1018B40075F00AA42441FF7D3711F7255BF8A620B3
:1018C400055B80D5D2AFD28C7536FF90E680E020E0
:1018D400E118E0440AF07FC47E091201A290E65D9B
:1018E40074FFF090E65FF05391EF538EF831373187
:1018F4001380FC7B0A11FE742122AE031BEE600EE2
:10190400AE050DA806E6AC070FA804F680EC22E4A9
:10191400F55CF55D90E6A3E020E21071FFEF700343
:10192400020492313090E6A3F0D2182290E6A67415
:1019340001F02290E6A0E04480F02290E6B8E0F5C1
:101944006F90E6BAE0F57090E6BCE0F57190E68A37
:10195400E4F074E090E6B3F0E56F5460600241F3A4
:1019640090E6B9E07002412E147002417E24FE70AC
:101974000241C124FB7002412714700241221470F9
:1019840002410E14700241152405600241F190E6F3
:10199400BBE024FE602614604124FD600B14602B20
:1019A400240670647163805890E6FBE06002613A3B
:1019B40074002498F58274E03400804490E680E05A
:1019C40030E70471588002714D803590E680E03034
:1019D400E704714D800271588026E570601875F037
:1019E40002A4FF7163FCEF2582FFE5F03CCF24F0F5
:1019F400CF34FFEF800E74002452F58274E034007B
:101A0400AF82E58291A56141613A90E740E52F619B
:101A14002D71437418F07438F085702F614185700E
:101A240030614190E740E530612DE56F247F60101F
:101A34001460152402704190E7407401F0A3802ED5
:101A440090E740E4F0A38027E571B4020590E6A393
:101A54008008E571B4880890E6A6E054018004E5A6
:101A640071700690E740F08002613A90E741E4F03B
:101A740090E68B7402F06141613AE56F24FE6004E4
:101A84002402613AE57070333018026141E571B4A3
:101A9400020C1211E5714390E6A3E4F06141E57193
:101AA400B4881090E6837418F07438F090E6A6E4D5
:101AB400F06141E57170026141807B8079E56F24BA
:101AC400FE600C24027024E570640260708067E597
:101AD400707016E571B4020590E6A38050E571B408
:101AE400880590E6A68046804D804B80498047E576
:101AF4006F54606420703F90E6B9E02402601B14C8
:101B04007032E56FB42111E571700D5391EF75A139
:101B140001C2AF1200038025801CE56FB4A113E558
:101B240071700FE5551490E740F090E68B7401F066
:101B3400800B8002800090E6A0E04401F021379001
:101B4400E6837402F07422F02274002412F5827485
:101B5400E034002274002432F58274E034002274EC
:101B6400002400F58274E0340022C0E0C083C08207
:101B7400C0D090E680E030E766757201757310900E
:101B8400E6FCE0640D601CE57315737002157214B5
:101B94004572600F90E6FEE030E3E4757200757301
:101BA400C180DC90E6FCE0B40C1590E6FB7402F016
:101BB400757400A3740DF075740090E6FBE4F07185
:101BC40058F583A37402F0714DF583A37407F0757F
:101BD4002D02752E0090E6367489F0A37490F0718E
:101BE400F45391EF75A120D0D0D082D083D0E032CD
:101BF400E52D90E626F0E52EA3F02290F000E0B467
:101C04005510A3E0B4530BA3E0B44206A3E064432D
:101C140060037F0122120F94641F4E7F0060027FD5
:101C24000122A28CB3921C75AF07759DFC301C0F6A
:101C34007EE07F007C017D007A007BA21205BCE47B
:101C4400F55AC218F555F520F522F521C21A1211DC
:101C5400797B801205B2758921758E10D2A9D28C38
:101C640022C0E0C0F0C083C082C0D075D000C000E4
:101C7400C001C002C003C004C005C006C007539120
:101C8400EF75A101313FD007D006D005D004D003B1
:101C9400D002D001D000D0D0D082D083D0F0D0E018
:101CA40032AC0774E0F59A8C9BE4FF90E67BE0FE8F
:101CB40074402FF582E434E7F583EEF00FBF40EB78
:101CC40090E6BBE064026004E0B4070790E742E0FA
:101CD400FD800590E740E0FD90E6BFE0701590E6DA
:101CE400BEE0FFEDC39F5004AF05800590E6BEE063
:101CF400FFAD0790E68BEDF022755A04B118A3E00E
:101D0400F52CA3E0F52BA3E0F52AA3E0F529A3E045
:101D140033921F2290F004E0F556A3E0F557A3E0B8
:101D2400F558A3E0F55922AE031BEE60130DED8CBC
:101D34008370010C14F582E0AA070FA802F680E76D
:101D440022D2215391EF75A108321207C7120FF75F
:101D5400D10A12178F1217BA121779552BFEE52CD8
:101D64005F4E60028044E52DC313FEE52E1324FF6D
:101D7400FFEE34FFFE90E6D0E0FCA3E0FDC3E56493
:101D84009DFDE5639C5EFEED5F4E6002801C7E005F
:101D940090E6CEE0FCA3E0B56218EEB50414A3E02F
:101DA400FEA3E0B5640CEEB56308D21990E648745E
:101DB40008F090E61B74051216C0701CE52C540143
:101DC400FF8F61A3E0FEA3E0FFE4FCFD78011200B5
:101DD4007AD101E561422CE4120756500D7F22129C
:101DE4000203BF4002D1187F012212001BEF30E32F
:101DF400037F0222E533600215337F00228F2C8E8D
:101E04002B8D2A8C292278011200678F648E638DB2
:101E1400628C6122740A2533F533C394144017E5A8
:101E24003CB44407753C42AF3C8005E4F53C7F0C70
:101E340012073AE4F533228E608F61E4F564F565A8
:101E4400C3E5659561E5649560504C90E6A3E02098
:101E5400E2F9E4F562F563C3E563952EE562952D39
:101E64005024E5652563FFE5643562FEE42563FDE2
:101E7400E56234F0FC7B10D19C74102563F563E4B7
:101E84003562F56280D112048BE52E2565F565E592
:101E94002D3564F56480A9228E668F678C688D6900
:101EA4008B6AD1FDF11FD1E8500122E566D1E450DF
:101EB4000122E567D1E4500122E56A601D0569E568
:101EC40069AE687002056814F5828E83E090E67945
:101ED400F0F12A500122156A80DFF117F105C322BF
:101EE40090E679F090E678E0FF30E0F8EF30E20237
:101EF400D322EFC320E101D32290E678E020E6F973
:101F040022D1FDF11FF12AF117D1FD90E678E030DE
:101F1400E1F12290E678E04440F02290E678748083
:101F2400F0A374A2F02290E678E0FF30E0F8EFC36B
:101F340030E201D322AF08EF3395E0FE75F003EFF2
:101F44001200A5EE75F003A42583F583E49390E6CF
:101F54007CF02274FE252AF52A74FF352922ECC36D
:101F64001390E6D0F07580A0ECC313ED13A3F02218
:101F7400A2AF9222C2AF1207FB7F017E000201A230
:101F8400E4F561F562F563F564F565F566F56722D8
:101F9400C3E52E9567FFE52D9566FEC3EF22E56543
:101FA4002567F567E5643566F566227CFC1205BC99
:101FB400E4F59E2290E67CF0740AF022750802E5AE
:0C1FC40008640222E0243090E67CF02249
:00000001FF
